:100000000C94DF070C9417080C9417080C94133405
:100010000C9417080C9417080C9417080C941708E4
:100020000C9417080C9417080C947A220C946821ED
:100030000C9418240C9417080C9417080C941708A7
:100040000C9417080C9417080C9417080C941708B4
:100050000C9417080C94AF230C9417080C941708F1
:100060000C9417080C9417080C9417080C94170894
:100070000C9417080C9417080C9417080C94170884
:100080000C9417080C9417080C9417080C94170874
:100090000C9417080C9417080C9417080C94170864
:1000A0000C9417080C9417080C941708220A170AC6
:1000B0002F0A390A410A000A4B0A060B140B190BC6
:1000C0001E0B230B280B2D0B320B370B3C0B410B5C
:1000D000480B4A0B4C0B4E0BBC0DBC0DBC0DBC0DA4
:1000E000BC0DBC0DC60BC60B070C070C320CAC0DBF
:1000F000530DAC0D4E0CE50CF60CF60CF61E1D1F48
:10010000B5201D1FB520651F881FB52077208A20C8
:1001100000040104020403040404050400050105AD
:10012000020503050405050500060106020603068F
:100130000406050600070107020703070407050771
:10014000000001000200030004000500000101019D
:10015000020103010401050100020102020203027F
:100160000402050200030103020303030403050361
:10017000000000000000000000000000000000007F
:10018000000000000000000000000000000000006F
:10019000000000007E0F00D4FFFFFFC700000078C2
:1001A00000000000000000002A2B280000000000D2
:1001B0000000000000000000000000290000000016
:1001C0002C1E3420212224342627252E362D373884
:1001D000271E1F202122232425263333362E37388D
:1001E0001F0405060708090A0B0C0D0E0F1011124B
:1001F000131415161718191A1B1C1D2F3130232D17
:10020000350405060708090A0B0C0D0E0F10111214
:10021000131415161718191A1B1C1D2F3130354CC5
:10022000716D6B20636F6D70696C65202D6B622042
:100230006B6C6F72202D6B6D2064656661756C74DC
:100240000000DA1281FFD9F1DB20A4A62EAF00A0B6
:10025000C0D30000A1C8D30000AED580A83F408D18
:10026000142000E1E1E1E1E1E1E1E1E1E1E1008F20
:100270009000939400E1E100919200A0A1A2A3A4B8
:10028000E100B7B800B5B6008081828384E100E167
:10029000E1E1E1E1E1E1E1E1E1E1E1E100979800A3
:1002A000959600C0C0C0C0C0C0C0C0C0C0C0C0C063
:1002B000C0C0C0C0C0C0C0C000000000000000003E
:1002C000000000000000000000000000000000002E
:1002D000000000000000000000F0F0F0F0FFFFFF61
:1002E000FFFFFFFFFFFFFFFFFFFFFFFFFFFFFFFF1E
:1002F000FFFFFFFFFFFFFFFFFFFFFFFFFFFFFFFF0E
:10030000FFFFFFFFFFFFFFFFFFFFFFFFFFFFFFFFFD
:10031000FFFFFFFFFFF0F0F0F00000000000000022
:1003200000000000000000000000000000000000CD
:1003300000000000000000000000000000000000BD
:1003400000000000000000000000000000000000AD
:10035000000000000000000000FFFFFFFFFFFFFFA4
:10036000FFFFFFFFFFFFFFFFFFFFFFFFFFFFFFFF9D
:10037000FFFFFFFFFFFFFFFFFFFFFFFFFFFFFFFF8D
:10038000FFFFFFFFFFFFFFFFFFFFFFFFFFFFFFFF7D
:10039000FFFFFFFFFFFFFFFFFF0000000000000066
:1003A000000000000000000000000000000000004D
:1003B000000000000000000000000000000000003D
:1003C0000000000000F0F0F0F0FFFFFFFFFFFFFF74
:1003D000FFFFFFFFFFFFFFFFFFFFFFFFFFFFFFFF2D
:1003E000FF0F0F0F0F00000000000000000F0F0FA5
:1003F0000FFFFFFFFFFFFFFFFFFFFFFFFFFFFFFFFD
:10040000FF0F0F0F0F00000000000000000F0F0F84
:100410000FFFFFFFFFFFFFFFFFFFFFFFFFFFFFFFDC
:10042000FFFFFFFFFFFFFFFFFFF0F0F0F000000015
:1004300000000000000000000000000000000000BC
:100440000000000000FFFFFFFFFFFFFFFFFFFFFFB7
:10045000FFFFFFFFFFFFFFFFFFFFFFFFFFFFFFFFAC
:10046000FFF0F0F0F00000000000000000F0F0F0FD
:10047000F0FFFFFFFFFFFFFFFFFFFFFFFFFFFFFF9B
:10048000FFF0F0F0F00000000000000000F0F0F0DD
:10049000F0FFFFFFFFFFFFFFFFFFFFFFFFFFFFFF7B
:1004A000FFFFFFFFFFFFFFFFFFFFFFFFFF00000059
:1004B000000000000000000000000000000000003C
:1004C0000000000000FFFFFFFFFFFFFFFFFFFFFF37
:1004D000FFFFFFFFFFFFFFFFFFFFFFFFFFFFFFFF2C
:1004E000FFFFFFFFFFFFFFFFFFFFFFFFFFFFFFFF1C
:1004F000FF0F0F0F0F0F0F0F0F0F0F0F0F0F0F0F1C
:100500000FFFFFFFFFFFFFFFFFFFFFFFFFFFFFFFEB
:10051000FFFFFFFFFFFFFFFFFFFFFFFFFFFFFFFFEB
:10052000FFFFFFFFFFFFFFFFFFFFFFFFFF000000D8
:1005300000000000000000000000000000000000BB
:1005400000000000000F0F0F0FFFFFFFFFFFFFFF76
:10055000FFFFFFFFFFFFFFFFFFFFFFFFFFFFFFFFAB
:10056000FFFFFFFFFFFFFFFFFFFFFFFFFF0F0F0F6B
:100570000F00000000F0F0F0F0F0F0F0F0000000EC
:10058000000F0F0F0FFFFFFFFFFFFFFFFFFFFFFF3A
:10059000FFFFFFFFFFFFFFFFFFFFFFFFFFFFFFFF6B
:1005A000FFFFFFFFFFFFFFFFFF0F0F0F0F00000018
:1005B000000000000000000000000000000000003B
:1005C000000000000000000000000000000000002B
:1005D000000000000000000000FFFFFFFFFFFFFF22
:1005E000FFFFFFFFFFFFFFFFFF0F0F0F0F000000D8
:1005F00000F0F0F0F0FFFFFFFFFFFFFFFFF0F0F073
:10060000F0000000000F0F0F0FFFFFFFFFFFFFFFC5
:10061000FFFFFFFFFFFFFFFFFF00000000000000E3
:1006200000000000000000000000000000000000CA
:1006300000000000000000000000000000000000BA
:1006400000000000000000000000000000000000AA
:10065000000000000000000000FFFFFFFFFFFFFFA1
:10066000FFFFFFFFFFFFFFFFFFF0F0F0F0F0F0F003
:10067000F0FFFFFFFFFFFFFFFFFFFFFFFFFFFFFF99
:10068000FFF0F0F0F0F0F0F0F0FFFFFFFFFFFFFFF2
:10069000FFFFFFFFFFFFFFFFFF0000000000000063
:1006A000000000000000000000000000000000004A
:1006B000000000000000000000000014001A000804
:1006C00000150017002B0004001600070009000A9F
:1006D000004C001D001B000600190005000000E092
:1006E00000427E2C00E200A8000000130012000C63
:1006F0000018001C00340033000F000E000D000B2A
:1007000000E5003800370036001000110000002A14
:1007100000437E2800E300AE00000014001A000928
:100720000013000A002B00042815241621172207A5
:100730000014001D001B0006001900050000004CFD
:1007400000427E2C002900E100000033001C00184C
:10075000000F000D00340012280C24082111320B68
:1007600000310038003700360010000E0000002A6B
:1007700000437E2800E300AE000000390053005221
:10078000002E002F0229004A00500051004F002F78
:100790000000004D004B0016014E00260200000133
:1007A00000010001000100A8000000570061006086
:1007B000005F00300234022D005E005D005C0030FE
:1007C00000010055005B005A00590027020000623A
:1007D00000010001000100AE0000001E021F022007
:1007E00002210222020000000000000000000000C0
:1007F00000000000000000000000000000000001F8
:1008000000010001000100A80000003100201418C0
:100810001424022302000000000000000000000079
:1008200000000000000000000000000000000001C7
:1008300000010001000100AE0000000000000023E4
:100840007821780000007C027C407E257800000042
:1008500000467E457E417E277800000000000001B2
:1008600000010001000100A80000006900420041F1
:100870000040000000680045003F003E003D0000D1
:1008800000440043003C003B003A0000000000012F
:1008900000010001000100AE0005010980A10185F1
:1008A0000319012AB700150126B7009501751081BB
:1008B00000C0050C0901A101850419012AA0021537
:1008C0000126A002950175108100C005010906A14D
:1008D00001050719E029E715002501950875018133
:1008E000029501750881010507190029FF150026E9
:1008F000FF009506750881000508190129051500F6
:100900002501950575019102950175039101C009B5
:10091000023B00020100A0FA0904000001030101EA
:10092000000921110100012244000705810308008C
:100930000109040100010300000009211101000167
:10094000223200070582032000011201000200008C
:1009500000083C3A01003001010200010A034B008B
:100960004C004F00520000000C03470045004900B6
:1009700053005400000004030904000000000000BC
:100980003E5B4F5B3E003E6B4F6B3E001C3E7C3E31
:100990001C00183C7E3C18001C577D571C001C5E38
:1009A0007F5E1C0000183C180000FFE7C3E7FF0053
:1009B000001824180000FFE7DBE7FF0030483A0684
:1009C0000E00262979292600407F05050700407F73
:1009D00005253F005A3CE73C5A007F3E1C1C08009E
:1009E000081C1C3E7F0014227F2214005F5F005F02
:1009F0005F0006097F017F00006689956A006060DC
:100A00006060600094B6FFB69400080C7E0C08008D
:100A100010307E30100008083E1C0800081C3E08FC
:100A200008001E10101010000C1E0C1E0C00303898
:100A30003E383000060E3E0E0600000000000000AA
:100A400000005F000000000700070000143E143E95
:100A500014002E2A7F2A3A00201208240200374967
:100A600049375000000807030000001C2241000025
:100A70000041221C00002A1C7F1C2A0008083E0896
:100A80000800008070300000080808080800000016
:100A9000606000002010080402007F5149457F007B
:100AA0000804027F0000714949494F00414149490A
:100AB00077000F1010107F004F49494971007E499F
:100AC00049497000010171090700774949497700D8
:100AD000074949493F00000014000000004034006D
:100AE00000000008142241001414141414000041E2
:100AF00022140800010159090F007F415D594F0080
:100B00007F0909097F007F49494976007F414141BA
:100B100041007F4141417E007F49494949007F09A9
:100B2000090909007F4141497B007F0808087F00CF
:100B300000007F000000704040407F007F080808F0
:100B400077007F40404040007F011F017F007F040D
:100B500008107F007F4141417F007F0909090F0094
:100B60007F4171417F007F0909196F004749494959
:100B7000790001017F0101007F4040407F001F207C
:100B800040201F007F407F407F00770808087700E3
:100B90004F4848487F00615149454300007F41412B
:100BA00000000204081020000041417F0000040200
:100BB00001020400404040404000000007080000DF
:100BC000605454547C007F44444478007C44444442
:100BD0004400784444447F007C5454545C00087FB3
:100BE0000909090038A4A4A4FC007F0404047800C7
:100BF00000007D0000007040407D00007F08080874
:100C0000760000007F4000007C047C047C007C04B3
:100C1000040478007C4444447C00FC2424243800F0
:100C200038242424FC007C04040404005C54545440
:100C3000740004047F0404007C4040407C001C20BD
:100C400040201C007C407C407C006C1010106C002C
:100C5000BCA0A0A0FC004464544C440000083641F1
:100C6000000000007700000000413608000002018B
:100C7000020402003C2623263C000000E0F0F0F0D5
:100C8000F0FEFF9F0F0F9FFFFFFFFF9F0F0F9FFFC4
:100C9000FEF0F0F0F0E00000FF000000000000C0F7
:100CA000300C0300000000FF000000000000000006
:100CB000E010080402020201010101010102020226
:100CC000040810E000000000FF0101010101010122
:100CD000010101FF7F515555457F415F5F5F7F00F7
:100CE0007F417B77417F415F5F5F7F007F415D5D3B
:100CF0005D7F415F5F5F7F00C0E0F0F0F0E0E6F70E
:100D0000F3F060007C7C7C7C7C007C7C7C7C7C00C8
:100D1000F81CDE1FFFFFFF1FDE1CF800C0E2B4F866
:100D2000F8F8F8F8B4E2C00000000000000000008D
:100D3000000000000000000000000000070F0F0F7F
:100D40000FFFFFFFFF9F87E1F9F9E1879FFFFFFF9B
:100D5000FF0F0F0F0F070000FF0000C0300C33C063
:100D600000000000000000FF000000000000003F45
:100D7000C0000000000000000000000000000000B3
:100D8000000000C03F000000FF08080808080838FD
:100D9000C808080F7E00007F00007800007E000079
:100DA0002424121224244848242412120000000093
:100DB00000000000000000000F1F3F7F7F3F3F7FCB
:100DC0007F3810001F1F1F1F1F001F1F1F1F1F0026
:100DD0000F1421404541454021140F007D7D7D7D4C
:100DE0007D7D7D7D7D7D7D00000000000000000098
:100DF00000000000000000000000080808080808C3
:100E000000000000000000000000000000000000E2
:100E100000000000000000003F0C03000000000084
:100E2000030C30000000003F202020202020202044
:100E30000102040810101020202020202010101083
:100E400008040201000000003F0000000000000054
:100E500000030C3040000040000040000040000053
:100E60001C3E3E3E1C003E1C1C0808003E3E3E3E12
:100E70003E00000000000000000000000000000034
:100E80000000000000000000000000000000000062
:100E90000000000000000000000000000000000052
:100EA0000000000000000000000000000000000042
:100EB0000000000000000000000000AF00AE0001D4
:100EC000010101010101010102020202020202020A
:100ED00002030303030303030304040404040404DC
:100EE00005050505050606060606070707070708A0
:100EF000080808090909090A0A0A0B0B0B0C0C0C53
:100F00000D0D0D0E0E0E0F0F0F10101111111212EC
:100F100013131414151516161717181819191A1A69
:100F20001B1B1C1D1D1E1E1F2020212222232424CA
:100F3000252626272829292A2B2C2D2D2E2F303106
:100F40003232333435363738393A3B3C3D3E3F4018
:100F50004142434445464748494A4C4D4E4F505103
:100F60005354555658595A5B5D5E5F6162646566BD
:100F700068696B6C6D6F7072737577787A7B7D7E44
:100F80008082838587888A8C8E8F91939596989A94
:100F90009C9EA0A2A3A5A7A9ABADAFB1B3B5B7BAAC
:100FA000BCBEC0C2C4C6C9CBCDCFD1D4D6D8DBDD80
:100FB000DFE2E4E7E9EBEEF0F3F5F8FAFDFF1124E8
:100FC0001FBECFEFDAE0DEBFCDBF04B603FE18C010
:100FD0008091520990915309A0915409B0915509FB
:100FE0008730904BA740B04B59F4109252091092A1
:100FF00053091092540910925509E0E0F8E309955D
:1010000012E0A0E0B1E0E0ECFCE602C005900D9239
:10101000AC3AB107D9F729E0ACEAB2E001C01D92C1
:10102000A235B207E1F70E94230E0C945E360C94B1
:101030000000A6E0B0E0EFE1F8E00C9457354983FA
:101040005A8349815A81992361F0222351F0CA01C0
:101050000E949B26182F682F89819A810E94C72899
:1010600004C0CA010E949428182F69817A81812FB7
:101070000E94CC172696E3E00C9473350E94292930
:101080002FEF84E39CE0215080409040E1F700C0C6
:1010900000009CE088E10FB6F894A895809360006A
:1010A0000FBE90936000FFCF8823B9F19CEF980F9B
:1010B000913A60F4E1E0F8E09281891301C0128274
:1010C000319648E0E730F407B9F714C090E2980F82
:1010D000983098F4877021E030E0A90102C0440FF5
:1010E000551F8A95E2F7CA0180959091650889237A
:1010F000809365080E94112608959BE5980F933010
:1011000028F480E090E00E9466240895885A8B318C
:1011100020F480E090E00E94412408950F931F93F3
:10112000CF93882309F465C0C82F8CEF8C0F813AC8
:1011300050F503E018E089E098E0F8012191C2172A
:1011400021F08E179F07D1F70EC0E1E0F8E087E0AD
:1011500098E02281C21301C0128231968E179F0738
:10116000C1F70E941126EFEF80E0D8019D918D011B
:10117000C917C9F0EF3F19F4911101C0E82F8F5F33
:10118000863099F72DC080E28C0F883078F4C770D4
:1011900081E090E001C0880FCA95EAF79091650858
:1011A000892B809365080E94112623C0EBE5EC0F84
:1011B000E33040F4F0E0E554FE4F808190E00E947F
:1011C000662417C0C85ACB31A0F4EC2FF0E0EE0F24
:1011D000FF1FE254FE4F808191810E94412409C08B
:1011E000EF3F09F30E2E000CFF0BEF5FF74FC283AA
:1011F000DACFCF911F910F910895ABE1B0E0E3E01A
:10120000F9E00C945435688F798F8A8F9B8FE42E88
:10121000152FF82E092F91111092640841E0F41255
:1012200046C0183008F043C085E08E1508F43FC072
:10123000612F70E02E2D30E0C901A6E01A9F800DCD
:10124000911D1124DC0143E0B695A7954A95E1F77D
:101250008770992741E050E0FA0102C0EE0FFF1FAE
:101260008A95E2F7CF01AA53BD4F002319F04091B0
:10127000220802C04C914E234423A9F096E0969F89
:10128000A001979F500D1124420F531F440F551F6B
:10129000FA01EF5EFE4F1491FA01E05FFE4FE49019
:1012A0009C91892B03C080959C9189238C93DE01AE
:1012B0001F9687E0FD0111928A95E9F7EE8A1F8B50
:1012C00086E0FE01769601900D928A95E1F7FF2067
:1012D00049F021E04E2D512F69897A898F2D902F69
:1012E0000E941908EF86188BFB8A0C8B87E0FE01A1
:1012F0003F96DE01189601900D928A95E1F7CE0196
:1013000008960E94FF2681113BC087E0FE013896B7
:10131000DE01119601900D928A95E1F76C856623A6
:1013200079F120912A0830E0C90101968770992748
:101330004091630850E084179507A1F06D8397E012
:10134000929FD001939FB00D1124A55DB74FFE0170
:10135000319601900D929A95E1F780932A080E94A8
:1013600038260EC00E94292910922A08109263087C
:10137000E3E2F8E087E0DF011D928A95E9F719C002
:1013800017E08091630890912A08891791F0189FBF
:10139000C0011124855D974F0E94FF26882349F0E4
:1013A0008091630890E00196877099278093630885
:1013B000E8CF6B96E6E00C947035A0E0B0E0E3EE89
:1013C000F9E00C944C35FC018481882309F4D4C3E2
:1013D0008F0121E0408151816281738195810E945A
:1013E00019086C01FC01E054FE47E730F10508F0F4
:1013F000FAC0EA5AFF4FD80115968C910C94193611
:10140000882309F4B9C38091F60280FD02C081608F
:1014100001C08E7F8093F6026091F5027091F60212
:1014200084E090E00E94D4350E942929A5C3882336
:1014300009F4A2C362E083E090E00E94B63582E046
:1014400090E00AC0882309F497C361E083E090E04C
:101450000E94B63581E090E00E9424298DC3882344
:1014600011F082E009C082E00E9402290E94D91D89
:1014700083C3882321F083E00E941429F7CF83E0FF
:10148000F3CF882321F084E00E94142975C384E0FF
:101490000E94022971C3882309F4A5C0C0E2D2E0EA
:1014A0005AE0652EFE012491222309F499C02130CF
:1014B00009F03DC031968491813021F42296FE01DD
:1014C000849188C0823031F42296FE0184910E947A
:1014D0008E0884C0833031F42296FE0184910E94EC
:1014E00054087CC0843009F078C02296FE01249113
:1014F00080E090E030E0205331092A30310560F47B
:10150000689EA001699E500D1124C901840F951F8A
:101510002196FE012491EECF009709F45FC0AFE958
:10152000BFE01197F1F700C000000197F5CFE22F5F
:10153000F0E0E056FE4F7490822F86958695869552
:1015400090E0FC01E057FE4FA4902770B12C022ED2
:1015500002C0B594A7940A94E2F7B1E0AB22BB2491
:10156000FC01E058FE4F8490912C022E02C095940D
:1015700087940A94E2F7E1E08E229924FC01E05975
:10158000FE4FE490F12C02C0F594E7942A95E2F71F
:10159000F1E0EF22FF24A114B10419F081EE0E94C2
:1015A0008E088114910419F086EE0E948E08872D12
:1015B0000E946C298114910419F086EE0E9454084F
:1015C000A114B10419F081EE0E945408E114F10451
:1015D00029F08CE20E946C2901C0EF01219662CFB4
:1015E00088E20E946C29D80115969C9191115AC0ED
:1015F000809165088272F601E052F847E531F10505
:1016000008F096C0E35AFF4F0C9419369091BC072E
:1016100081E089278093BC07109255018091AA032D
:1016200081608093AA03A8C249E651E363E771E3AE
:101630002CC043E751E369E671E327C045E551E378
:101640006FE571E322C04FE551E365E571E31DC02D
:101650004BE351E368E471E318C048E451E36BE302
:1016600071E313C041E251E36EE271E30EC04EE25A
:1016700051E361E271E309C049ED50E367EE70E3C5
:1016800004C047EE50E369ED70E30E94772574C211
:1016900081E005C084E003C08CE001C080E10E94CD
:1016A000E91D6AC221E0C2162CE7D20609F43EC049
:1016B00033E0C3163CE7D30699F1C1144CE7D406D6
:1016C000B9F50E9429295FEF84E39CE051508040E6
:1016D0009040E1F700C0000081E08093E00080E2EC
:1016E0008093D8001092C900AFE1BEE41197F1F7E2
:1016F00000C0000087E090EBDC01809352099093DA
:101700005309A0935409B09355099CE088E10FB6A2
:10171000F894A895809360000FBE90936000FFCF6F
:101720006FEF7FEF80E090E00E94D4350E943E088A
:10173000F801C081D181992349F0CE010E949B26F6
:10174000F82E682FCE010E94C72804C0CE010E9447
:101750009428F82EBE018F2D0E94CC170E94E91705
:10176000D82FC82FF8012581368132953F70E92E98
:10177000E2944FE0E4224E2D50E04C30510508F049
:10178000EBC1FA01EE58FF4F0C941936892F807F78
:101790009F70F92E882319F0F29480EFF82222230B
:1017A000C9F0FF2009F46AC180E28D0F883010F083
:1017B000C11107C090916508C92FCF29C093650852
:1017C00006C090916408C92FCF29C09364080E9475
:1017D000112654C18D2F0E945408FF2009F4BCC16A
:1017E000D05E8F2D8095D83010F0C11107C0909138
:1017F0006508C92FC823C093650806C09091640886
:10180000C92FC823C09364080E941126A5C1492F7F
:10181000407F892F8F70403211F08295807FC130D8
:1018200051F4222321F0363008F096C108C035303B
:1018300008F092C114C0222329F031111FC10E9467
:101840004A298AC1332359F0D93309F028C1FFEF5F
:1018500027EE33E0F15020403040E1F71EC10E94F6
:101860003F297AC1892F86958695837019F081303A
:1018700059F072C1222319F08D2F937002C080E0BD
:1018800090E00E9466246EC1222319F08D2F937080
:1018900002C080E090E00E94412464C1892F8370DF
:1018A00009F046C021115CC18D2F82958695877005
:1018B000880F880F6D2F6F7070E0082E02C0660FC2
:1018C000771F0A94E2F7D4FF0BC04FE050E002C04C
:1018D000440F551F8A95E2F79A012095309502C072
:1018E00020E030E09695969593709230A9F0F0F450
:1018F00040916E0850916F08913031F0CB01822BEE
:10190000932B8423952305C0CB01842B952B822B0D
:10191000932B0E94242924C1CB01822B932B20914D
:101920006E0830916F0882279327F3CFCB01EFCF5A
:10193000222319F0892F817001C08695882309F42C
:101940000FC18D2F829586958770880F880F6D2F18
:101950006F7070E0082E02C0660F771F0A94E2F7DE
:10196000D4FF0BC04FE050E002C0440F551F8A95D2
:10197000E2F79A012095309502C020E030E096957C
:1019800096959370923089F0D0F44091AB035091CA
:10199000AC03913031F0CB01822B932B8423952320
:1019A00011C0CB01842B952B0BC0CB01822B932B29
:1019B0002091AB033091AC038227932703C0CB0166
:1019C000822B932B0E94FB28CBC0C92FCF702223E0
:1019D00039F08C2F0E9414298D2F0E944A29C0C0F3
:1019E0000E943F298C2F0E940229BAC0813F11F129
:1019F00018F4803F31F03EC0823F19F1833F41F13E
:101A000039C0222399F0353008F0A6C0292F2F7154
:101A100081E090E002C0880F991F2A95E2F720919B
:101A2000AB033091AC038227932721C0363008F0F6
:101A300093C0ECCF222339F0892F8F710E94142993
:101A40008BC02223C9F3892F8F710E94022984C081
:101A5000222359F09F7121E030E0A90102C0440F18
:101A6000551F9A95E2F7CA0102C080E090E00E94FB
:101A7000FB2872C0222331F03323F1F28D2F0E9414
:101A80008E086AC03323F9F2893349F45FEF87EE99
:101A900093E0515080409040E1F700C000008D2F4E
:101AA0000E94540859C0823FB1F028F4803F49F0A9
:101AB000813FF9F028C0843FB9F058F0853F71F0BC
:101AC00022C0222309F44EC09091220881E0892788
:101AD00008C081E028272093220844C0211142C079
:101AE00081E0809322083EC021113CC01092220860
:101AF00039C0222329F080912108882329F329C0A5
:101B0000353010F32FC0809121083323C1F0882392
:101B100041F09091220881E0892780932208109259
:101B200021088D2F222319F00E948E081BC00E94CD
:101B3000540887E0D8011D928A95E9F713C08823DD
:101B400089F021110FC09091220881E089278093AC
:101B500022081092210806C088EF8E0D843010F400
:101B60000E948B2420E0F8014081518162817381C1
:101B7000848195810E941908CDB7DEB7EEE00C9400
:101B80006835CF93DF93EC018091AB039091AC0368
:101B900020916E0830916F08282B392B832F9927BD
:101BA000009719F09C0198E001C090E0A90174E051
:101BB000569547957A95E1F74115510511F09C5FCF
:101BC0009A01A90156954795569547954115510596
:101BD00011F09E5F9A0136952795232B09F09F5FA0
:101BE000923091F038F4992361F0913099F46BE6DA
:101BF00071E012C0933059F0943061F463E871E001
:101C00000BC06EE571E008C067E771E005C06DE7E5
:101C100071E002C06AE871E08EEA92E00E945736F5
:101C20006EEA72E087EF92E00E945736CE018C7028
:101C300099270C9719F4CE01806102C0CE018F7EE6
:101C4000DF91CF910895A4E1B0E0E9E2FEE00C94C9
:101C5000483585B7806885BF85B7806885BF84B7FC
:101C6000877F84BF0FB6F894A89580916000886143
:101C700080936000109260000FBE90E080E80FB685
:101C8000F89480936100909361000FBE80E794E127
:101C90009093AD028093AC020E94AC210E941F225F
:101CA0008091E20084608093E20078948091A003A8
:101CB0008823A1F01091E9001F709091EC00892F0A
:101CC000817090FD80E8182B1092E9008091E80067
:101CD00083FD0E94151E1F701093E90082E084BDF1
:101CE00093E095BD9AEF97BD80936E001092CC0261
:101CF0001092CD021092CE021092CF028091D800A5
:101D000080618093D8002AE12A95F1F700C0809184
:101D1000D900182F117080FD04C00E94AC211092D0
:101D2000A0031093F3071093F4071093000111110F
:101D30000E94CE339091000181E098279093F102A8
:101D4000382F391B3093D102909100018093F20219
:101D5000909100018093D00280910001811106C012
:101D600084EF80930C0185EF80930B0180910C012F
:101D7000E82FE295EF70F0E041A1282F2F7081E06D
:101D800090E0BC0102C0660F771F2A95E2F79B0125
:101D9000362F3095342331A332A1232B22A3209157
:101DA0000B01E22FE295EF70F0E031A12F7001C03E
:101DB000880F2A95EAF7982F9095932391A392A1E3
:101DC000892B82A38FE891E00197F1F700C0000012
:101DD0007091F20203EF12E0ACE0B1E04BE051E0B1
:101DE00060E0671751F12D91822F82958F7090E0FE
:101DF000FC0180A190E02F7002C0959587952A95EF
:101E0000E2F78170FA019191AF01292F22952F708D
:101E100030E0F90120A130E09F7002C03595279590
:101E20009A95E2F720FD02C090E001C092E0892B74
:101E3000F80181938F016F5FD4CF80910001809171
:101E40000001811102C094E001C090E09093DB0298
:101E500084E0891B8093DA0201E911E0D8018D91B9
:101E60008D018F3F11F00E945317B1E005391B0718
:101E7000A9F705E911E0F80181918F018F3F11F079
:101E80000E945317F1E00B391F07A9F788E0ECED2A
:101E9000F2E0DF01282F1D922A95E9F7E2EDF2E04A
:101EA000DF011D928A95E9F780E090E00E94A0355D
:101EB000863E9E4F11F00E94A12582E090E00E9494
:101EC00098358093E40284E090E00E94A0359093DE
:101ED000F6028093F50283E090E00E94983590E04E
:101EE0000E9424298091AB039091AC030E94C10D04
:101EF0000E94D6301092C407EDEDF7E08FEF9FEF10
:101F00008193919327E0ED3EF207D1F71092A50857
:101F1000EEEBF8E08EEC98E02FEF3FEF219331935A
:101F20008E179F07D9F780E090E00E94A035863E8B
:101F30009E4F21F00E94A1250E94772F81E080937F
:101F4000AA0348E050E068E170E08CEB97E00E9463
:101F500088351092AA038091BC078C7F11F40E94EF
:101F6000772F82E080934F0380E88093AD030E9437
:101F700084326BE070E088E592E00E940C258823B3
:101F800009F443C080914F0365E070E081FD3AC0E1
:101F900083E592E00E940C258823B9F16DE070E0A2
:101FA00081E492E00E940C25882379F10E940024AC
:101FB000DC01CB01805A9541AF4FBF4F8093ED07B5
:101FC0009093EE07A093EF07B093F007E0EBF3E0F8
:101FD00080E094E0DF019C011D9221503040E1F748
:101FE000F093B707E093B6078FEF9FEF9093AF039F
:101FF0008093AE0381E08093F2078093F107109203
:10200000500303C08EE492E0C5CF8091F3078111A5
:1020100002C00E94D13381E091E09093F807809351
:10202000F7078091A003853009F055C030E4F32E06
:1020300000E112E18091A003853009F042C0809157
:10204000A003843069F181E00E947E310E94AC31AE
:1020500081E00E947E310E9437251092FB0748E103
:1020600050E00FB6F894A895409360000FBEF09230
:10207000600083B7817F846083BF83B7816083BF43
:102080007894889583B78E7F83BF0FB6F894A89510
:1020900080916000886180936000109260000FBEA4
:1020A00080919F03882309F4C5CF0E940C19ECEDA1
:1020B000F2E081918111FEC352E0E43EF507C9F7D9
:1020C000B9CF0E9429290E948B2480E00E947E3192
:1020D00080E00E947E310E940C1965EE72E07987E3
:1020E00068878CED92E0998B888BDC01FB019191E4
:1020F0008D9189272DEE32E02E173F0719F08823A6
:10210000B1F306C0811104C00E947629D12C64C1AC
:102110003091F3073A8B45E758E05B874A8766EFD3
:1021200071E07D876C87F12CA889B9897D90B98B86
:10213000A88BE885F985C080C724CF86CC2009F418
:1021400031C1CA84DB844C845D84E12CF1E0FF83DF
:102150008F852F81822309F415C1822E87203A8929
:102160003323A1F0E982FA820E940C249C838B83A2
:1021700041E04D8391E0811001C090E09E83498150
:102180005A816B817C818D810E94FD08882021F01D
:10219000D2018C918F3F11F4912C03C08E8799242A
:1021A0009394092D10E08091A508F801E80FF11D26
:1021B0003997ACF188E0A82EB12CA01AB10AB80169
:1021C0006F5F7F4F6B55774FA50186EA98E00E94BD
:1021D0004E36B801675F7F4F6B55774FA5018EEA8A
:1021E00098E00E944E36A501440F551FB801660FB6
:1021F000771F675E7F4F6B55774F8EEB98E00E949D
:102200004E36B8016F5E7F4F6B55774FA50186EB59
:1022100098E00E944E3688E089198093A508809145
:10222000A50890E0FE85AF2FB0E09D01220F331F7F
:102230002A5D3D4FAA0FBB1FBD01695D7D4F41E087
:10224000480F9915B0F490E0FC01EB55F74FD90118
:102250005C915183DB015C915187BE85B18B880F06
:10226000991FFC01EB55F74F128E118E91E0842FD0
:10227000E6CF8093A508882009F484C08091BC072C
:102280008C7F803609F07EC0F20180818F3F09F497
:1022900079C076EFA72E71E0B72EE5E78E2EE8E045
:1022A0009E2E612C282E312CC101880F991F9C0174
:1022B0002A5D3D4F3C8B2B8BC101880F991FAC01D0
:1022C000495D5D4F1A0100E010E0F501E00FF11FDC
:1022D00080818F3F09F446C06F100AC0E01208C029
:1022E000D6012C9130E2230F08F42FEF2C933AC043
:1022F00090E0EB89FC89408150E0FC01EE0FFF1F6C
:10230000EA5DFD4F2081421B5109D1012C9130E043
:10231000880F991FFC01EA50FE4F81A9281B310943
:10232000449FB001459F700D700D1124229FC00184
:10233000239F900D900D1124860F971F0E94D72F79
:10234000893280F428E2382F231B08F420E0F401BE
:10235000E00FF11F213108F020E13081320F08F445
:102360003FEF30830F5F1F4F0630110509F0ADCFEF
:10237000639446E0840E911C56E0A50EB11C68E003
:102380006612A1CFE3947F81770F7F838FEF481A86
:10239000580A9FEFC91AD90AA6E0EA12D9CEE885F1
:1023A000F9857082F394288539852F5F3F4F3987EF
:1023B00028874C855D854A5F5F4F5D874C876A85BE
:1023C0007B856A5F7F4F7B876A8778E0F712ACCEA8
:1023D0000E946A17DD24D3940E94AC31E12CC12CF9
:1023E0008091F202E81608F083C00E2D10E0F8018B
:1023F000E45FFE4F8081E82FE295EF70F0E0E0A10E
:10240000F0E08F7002C0F595E7958A95E2F7E170EC
:10241000D801A55FBE4F2C91A22FA295AF70B0E05E
:1024200090968C9190E02F7002C0959587952A9593
:10243000E2F780FD02C080E001C082E04E2F482B11
:10244000D801AD50BD4FEC918E2F837090E0242FBA
:10245000042E000C330B8217930709F447C0EE0FCC
:10246000EE0FE42BEC93F090F102FE0CEF70F0E035
:10247000E556FE4F01511D4F9081D8018C91890F77
:102480008C93823084F0EF2DF0E0E351FD4F80819A
:102490008F5F80838091F307882339F060E08F2D70
:1024A0000E94B32402C020E001C021E0F801808135
:1024B0008F3F84F4EF2DF0E0E351FD4F8081815098
:1024C00080838091F307882321F061E08F2D0E94A3
:1024D000B32421E0D8018C91082E000C990B62E006
:1024E00070E00E94E635F8018083C22AE39478CF39
:1024F000CC2021F00E949E25DD24D3948091F20708
:10250000882309F4C8C180915103909152030E941D
:10251000F123C29708F4B6C00E940C249093520392
:102520008093510380EB93E09093B7078093B607B5
:102530008091F307882309F47CC0E7EFF2E0019073
:102540000020E9F78F010150110987EFE82E82E0A2
:10255000F82EE016F10630F4D7018D917D010E942E
:102560004C1DF7CF81E00E94DC2483EA92E00E94B8
:10257000CB1D81E00E94DC248091F60280FF03C025
:1025800080EA92E002C08DE992E00E94CB1D8FE8C4
:1025900092E00E94CB1D88E892E00E94CB1D8091C2
:1025A000F60280FF03C085E892E002C082E892E074
:1025B0000E94CB1D8FE892E00E94CB1D8BE792E03A
:1025C0000E94CB1D83EA92E00E94CB1D81E00E9415
:1025D000DC240E948B2481FB002700F982FB112759
:1025E00010F980FF03C088E792E002C085E792E01F
:1025F0000E94CB1D002319F082E792E002C085E71C
:1026000092E00E94CB1D112319F08FE692E002C0E8
:1026100085E792E00E94CB1D83E692E00E94CB1DED
:1026200085E792E00E94CB1D85E792E00E94CB1DDA
:1026300029C02091AE033091AF03A0EBB3E080E05E
:1026400090E0FC01E754FD4FE4914C91E41781F0D8
:10265000EC93AC0116E0569547951A95E1F7E1E049
:10266000F0E002C0EE0FFF1F4A95E2F72E2B3F2B42
:10267000019611968115F4E09F0719F73093AF0387
:102680002093AE038091AE039091AF03892B31F478
:102690008091F107882309F4FEC0E6C08091F2071B
:1026A0008823B1F3809150038111F2CF0E9451250C
:1026B0002091AE033091AF032115310549F380E03D
:1026C000082F10E0EE24E394F12C082E02C0EE0C4B
:1026D000FF1C0A94E2F7A70142235323452B11F470
:1026E0008F5FEECF90914F039801F6E0220F331FDA
:1026F000FA95E1F790FF13C0E6E036952795EA9545
:10270000E1F7220F220F220F20930F0110921201E6
:10271000295F2093100187E08093130112C0220FDC
:10272000232F221F330B31958295880F880F8074D9
:1027300080930F0120931201815C809310012093FC
:10274000130124E630E047E050E06DE071E088E7F7
:102750000E942C33892B09F09BCF80914F0380FF7F
:1027600063C080E4EFE0F3E0DF011D928A95E9F7B2
:10277000A80136E0440F551F3A95E1F763EB462E6A
:1027800061E0562E0BEA11E0F20181912F01D80190
:102790009D918D01BA01690F711D60557C4F90E0CC
:1027A000815F9C4FFC0127E0922E9F01281B390B73
:1027B0007724739401C0770C2A95EAF75B01812C8A
:1027C000D501CD905D01C720292D28192770622ED3
:1027D000022E000C330BBC2D01C0BB0F6A94EAF72C
:1027E0006B2E3195219531092770332701C0C6948E
:1027F0002A95EAF76C28C0806C286082839428E0D0
:102800008212DECF9A9431963FEF9312CECF6BEBCC
:10281000461661E0560609F0B7CF04E610E020E462
:1028200030E04FE053E00CC0A80186E0440F551F94
:102830008A95E1F740555C4F04E610E020E430E073
:1028400060E488E70E944D33892B09F021CFE094A2
:10285000F0948091AE039091AF03E822F922F092B8
:10286000AF03E092AE0314CF0E9400240091ED0765
:102870001091EE072091EF073091F007DC01CB01BA
:10288000801B910BA20BB30B8F3F9F4FAF4FBF47E6
:1028900010F40E943725D1100E9451250E948B24EC
:1028A00090915303891709F4BCCB809353030E9482
:1028B0000024B7CB09BD19BD09B400FEFDCF80913E
:1028C000D8008F7D8093D8008091E0008260809353
:1028D000E0008091E00081FDFCCF0E942929AACB75
:1028E00080E008959091F50292FF10C041E0282FFA
:1028F0002471243009F040E031E0282F287128307D
:1029000009F030E0431711F02CE0822793FF10C04C
:1029100041E0282F2471243109F040E031E0282FD4
:102920002871283109F030E0431711F02CE082279C
:102930003091F60230FF10C051E0282F2171213074
:1029400009F050E041E0282F2871283009F040E0DC
:10295000541711F029E0822731FF10C041E0282FE1
:102960002171213109F040E031E0282F2871283110
:1029700009F030E0431711F029E0822794FD877EAB
:1029800008958238910569F1B0F48133910509F415
:1029900075C048F48932910509F467C08A329105FF
:1029A00009F471C008958533910509F459C089333C
:1029B0009105B9F00895833E910589F138F4803E80
:1029C0009105D1F0823E910529F10895863E910549
:1029D000C9F1873E9105D9F1843E910509F06CC09B
:1029E00027C02091F50220FD57C021FD55C0209140
:1029F000F60223FD5BC008958091F50280FD48C07A
:102A00008091F60280FF48C08091F50284FD46C0A7
:102A100083EE51C08091F50282FF3CC0F5CF8091DA
:102A2000F50282FD37C08091F60280FD35C0ECCF03
:102A30008091F60281FF36C08091F50284FD2EC0A0
:102A400087EE39C08091F50283FF2AC0F5CF8091CF
:102A5000F50283FD25C08091F60281FD23C0ECCFF5
:102A60008091F50285FD22C01FC08091F50285FD91
:102A70001BC08091F60283FF19C00AC08091F50245
:102A800086FD16C017C08091F50286FD13C010C0E8
:102A900089E311C082EE0FC080EE0DC080E00BC054
:102AA00086EE09C084EE07C085E305C089E203C055
:102AB0008AE201C081E390E00895A0E0B0E0E3E69F
:102AC000F5E10C9450357C015B016A018091930320
:102AD0008A3018F001E010E002C00AE010E0C1E026
:102AE000D0E0B501C701F6010995811115C0219605
:102AF0000C171D0794F0CC9F9001CD9F300D300D29
:102B0000112480E090E045E34A95F1F7000001963A
:102B100082179307C1F7E5CF81E0CDB7DEB7EAE0D2
:102B20000C946C35A0E0B0E0E8E9F5E10C94523586
:102B3000C82F7B01D42F6901FB01608171818281E3
:102B400093810E94D523643671058105910510F4A7
:102B5000DD2339F10C2E000CDD0B01151105A9F058
:102B6000FE0183E0EE0FFF1F8A95E1F7EC5EFE4F5A
:102B70008181928182599C4F408150E00417150752
:102B800008F4A801B6010E944E36CE010E94B93465
:102B9000882341F00E940024F701608371838283BF
:102BA000938381E0CDB7DEB7E8E00C946E35A1E009
:102BB000B0E0EDEDF5E10C9456358091F107898395
:102BC0002091860330E090E041E02817390709F4AE
:102BD00040E001E010E09E012F5F3F4F6FE873E09F
:102BE00087E00E9492152196E4E00C947235A9E0EA
:102BF000B0E0EDEFF5E10C94563588E0ECEBF7E052
:102C0000DE01119601900D928A95E1F78091D2082C
:102C1000898749E050E06DE773E0CE0101960E949C
:102C2000413641E0892B09F440E009E010E09E01C3
:102C30002F5F3F4F6BE873E086E00E949215299664
:102C4000E4E00C9472350F931F93CF93DF93EC0164
:102C500044E050E063E773E00E94413641E0892B95
:102C600009F440E004E010E09E0166E673E082E0D3
:102C70000E949215DF91CF911F910F910895A1E0CD
:102C8000B0E0E5E4F6E10C944C35C62E4A0159015A
:102C9000682E880F7708C3010E94B934882309F48D
:102CA00066C0C30123E0880F991F2A95E1F7FC0154
:102CB000EC5EFE4F438150E04115510511F041E0BB
:102CC00050E0FC01EC5EFE4F6481758162597C4FDF
:102CD000CE0101960E944E36F4016081718182819D
:102CE00093810E94D523643671058105910538F4DE
:102CF000B701C8010E949C2499818917D1F10C2C3D
:102D0000000CDD08C6010E94B934782E8823E1F05A
:102D1000E114F104C9F0960183E0220F331F8A9574
:102D2000E1F7F901EC5EFE4F438150E0E416F50651
:102D300008F4A701F901EC5EFE4F648175816259C8
:102D40007C4FC5010E944E36B701C8010E949C24E9
:102D500091E02981281390E0D92ED72089F00E9494
:102D60000024F401608371838283938309C0D12C92
:102D700002C0DD24D394A701B801C5010E944E36DC
:102D80008D2D2196EEE00C946835A1E0B0E0EBECDF
:102D9000F6E10C945135EE24E394F12C08E713E0AE
:102DA0009E012F5F3F4F4AE653E064E083E00E94BC
:102DB0003F16B82E882309F43DC000E080E09091D2
:102DC000D0020917A0F5D090D102D00E2D2D30E001
:102DD000A90143515D4F7A01E1E0F0E0EC0FFD1FE6
:102DE000E00FF11D1081FA019081191BC12E1C14F6
:102DF0005CF4CA94F70180818F5F808360E08D2D41
:102E00000E94B32481E0F3CF912F17FD90E0191BAE
:102E1000112359F01F5FF70180818150808361E0A9
:102E20008D2D0E94B32481E0F3CF0F5FC8CF8111B5
:102E30000E949E258B2D2196E9E00C946D35A4E02F
:102E4000B0E0E5E2F7E10C9452356B0184E0E82E46
:102E5000F12C0FE613E09E012F5F3F4F42E653E057
:102E600061E080E00E943F16882361F049815A8129
:102E70006B817C8140935E0350935F03609360039A
:102E80007093610340915E0350915F036091600312
:102E900070916103F60140835183628373832496AA
:102EA000E8E00C946E35F894E82FE295EF70F0E0CE
:102EB00031A1282F2F7081E090E001C0880F2A9562
:102EC000EAF7982F9095932391A392A1892B82A33F
:102ED000789408950F931F938091F307882319F036
:102EE0000E9400240EC00E9400240091CC02109188
:102EF000CD022091CE023091CF02600F711F821F50
:102F0000931F1F910F910895A4E0B0E0EAE8F7E164
:102F10000C945835609187037091880380918903E0
:102F200090918A030E94D52364367105810591052D
:102F300070F10E946A17DC01CB010296A11DB11D40
:102F400089839A83AB83BC8380913D0190913E013C
:102F500082599C4F40913C0150E04530510510F0A2
:102F600044E050E0BE016F5F7F4F0E944E3685E027
:102F700090E00E94B934882359F00E9400246093A5
:102F80008703709388038093890390938A0381E079
:102F90002496E2E00C9474357830B0F46630A0F4F6
:102FA0008530A0F490E3899FF001112486E0789F9A
:102FB000E00DF11D1124E60FF11DEE0FFF1FE75488
:102FC000F94F85919491089580E001C081E090E0EF
:102FD00008951F93CF93DF930E94C114EC01C11594
:102FE00080E5D807E8F5C11590E4D90708F0ADC031
:102FF000C03ED10530F5CD3CD10508F099C0C83AA6
:10300000D10578F4C53AD10508F088C0C130D105A2
:1030100009F481C008F4F8C0C430D10508F0F7C045
:10302000F3C0C33CD10508F0EFC0C85AD0E0CC0FC4
:10303000DD1FC254DE4F0990D881C02DCE019464AB
:10304000E7C0C11580E2D80708F0D1C0C11591E0F2
:10305000D90708F070C0C83ED10508F4D8C0D4C064
:10306000C03682E5D80728F5C03492E5D90708F0C4
:103070007FC0C03282E5D80708F071C0C11592E563
:10308000D90708F487C04C2F4695469580E2489FA3
:10309000A0011124C37021E030E0C90102C0880FF3
:1030A000991FCA95E2F7EA01C82BD92BCE019D687A
:1030B000AFC0C03C82E5D807E0F4C03A92E5D9073A
:1030C00008F083C0C03882E5D80708F09DC08C2F77
:1030D0008F718695869590E2899F90011124C37027
:1030E00081E090E002C0880F991FCA95E2F79A68C4
:1030F00069C0C03E92E5D90708F471C0CE0196556B
:103100008F3F910511F008F07FC0CE0199270E94F2
:10311000C11490667DC081E090E07AC0C55AD0E0CD
:10312000C554DE4F8881C82FD0E0CE01906470C0B6
:10313000CE0190656DC08D2F0E947214182FCE01A4
:1031400099270E94C1141F715DC0CE0199270E946A
:10315000C114CC27DF70D06A8C2B9D2B59C0CF7146
:103160008C2F90E0D82FCC27CE01816F906A50C071
:103170008C2F8F718695869590E2899F90011124FE
:10318000C37081E090E002C0880F991FCA95E2F7F2
:103190009C6818C08C2F8F710E94721495E0D69590
:1031A000C7959A95E1F7CF70D0E0DC2FCC27282F78
:1031B00030E084FF05C084E0220F331F8A95E1F7D9
:1031C000D069CE01822B932B23C08C2F8F710E944C
:1031D00072148F71C82FD0E09C2F882719C0CF712F
:1031E000DD27DC2FCC27CE01806F906A11C08D2F98
:1031F0008F710E947214182FCE0199270E94C1145A
:103200001F719062912B04C080E090E001C0CE015C
:10321000DF91CF911F910895ACE0B0E0E2E1F9E1D8
:103220000C944B35AE014F5F5F4F7A0188E0DA01B5
:103230001D928A95E9F701E911E06A0185E9682E96
:1032400081E0782EAA24A394B12C2BE9822E21E0D0
:10325000922EF80180818F3F09F440C0F894E82F46
:10326000E295EF70F0E021A18F70A50102C0440F3C
:10327000551F8A95E2F7CA01922F982B91A392A12C
:103280008095892382A3789400C0E5E9F1E0512C70
:1032900031E021912F3F89F0A22FA295AF70B0E0CD
:1032A00090968C9190E02F7002C0959587952A9505
:1032B000E2F780FD02C0832F01C080E0582A330F5F
:1032C0008E169F0631F7D8018C918F3F11F00E9426
:1032D0005317B0EABA95F1F7F60150820F5F1F4F0E
:1032E000FFEFCF1ADF0A6016710609F0B2CF48E08F
:1032F00050E0B70182ED92E00E944136892B99F0AF
:1033000088E0F701A2EDB2E001900D928A95E1F715
:1033100081E0809356030E940C2490935503809380
:103320005403F12C27C0809156038823D1F30091D8
:10333000DB0280915403909155030E94F12305977D
:1033400080F310E004521D4F44E050E062ED72E063
:10335000C8010E944136892B09F426C184E0E2EDC0
:10336000F2E0D80101900D928A95E1F7FF24F394E1
:10337000109256038091F307E091DB02882309F451
:1033800096C019861A861B861C860E2F10E00452E2
:103390001D4F809193038A3060F44FE157E1BE01E5
:1033A000675F7F4FC8010E945D15882309F451C0F3
:1033B0000AC080915703909158030E94F123843FE3
:1033C000914058F757C043E256E1BE01675F7F4F17
:1033D000C8010E945D158823E1F145EC56E1BE016C
:1033E000675F7F4FC8010E945D15882391F144E813
:1033F00057E1BE01675F7F4FC8010E945D158823BA
:1034000041F147EF55E1BE01675F7F4FC8010E9460
:103410005D158823F1F047ED55E1BE01675F7F4FF1
:10342000C8010E945D158823A1F01092930380913A
:10343000DA0290E044E050E0BE01675F7F4F8452C3
:103440009D4F0E94413621E020935D03892B01F5B9
:10345000A5C0809193038F3F19F08F5F80939303F2
:10346000809193038A3018F30E940C2490935803A0
:103470008093570380915D03882309F48FC0FE0178
:10348000399684E0DF011D928A95E9F710925D0379
:10349000E091DA02F0E0E452FD4F89859A85AB8530
:1034A000BC8580839183A283B38381E078C000913F
:1034B000DA0210E004521D4FF0E0E452FD4F84E0C8
:1034C000AFE6B3E001900D928A95E1F764E070E019
:1034D0008FE693E00E949C2480936E0384E0E3E7F0
:1034E000F3E0D80101900D928A95E1F74091F20244
:1034F00050E06091F10270E063517D4FCE0109967A
:103500000E944E3689858093780361E070E0CE0199
:1035100009960E949C248093770380907903909071
:103520007A03A0907B03B0907C0380915903909123
:103530005A03A0915B03B0915C0388169906AA0612
:10354000BB06B1F08092590390925A03A0925B039C
:10355000B0925C030E940024861A970AA80AB90A4E
:103560008092CC029092CD02A092CE02B092CF0275
:1035700088E0EDE7F3E0ACEBB7E001900D928A95BF
:10358000E1F7809185030E947E3180918603882334
:1035900019F00E94512502C00E94372580E08F2932
:1035A0002C96EFE00C946735F12CE2CE2F923F92EF
:1035B0004F925F927F928F929F92AF92BF92CF92E3
:1035C000DF92EF92FF920F931F93CF93DF93CDB7CC
:1035D000DEB72B970FB6F894DEBF0FBECDBF9D832D
:1035E0008C83809156010E949831292E582E20916B
:1035F000C4072B83521408F084C0A52CB12CF5010C
:10360000E658FD4F908180915701892309F477C0D6
:103610003090BD074090BE0784EC882E87E0982E3E
:103620008DED97E09A83898310E0712CC501880F96
:10363000991FFC01EA5DFD4FFF83EE83C501880FF2
:10364000991F9C01295D3D4F39872887FFEF8F1A0D
:103650009F0A2B81271509F442C0EE81FF81F0817A
:103660002F2F30E0F4018081281B31093B872A8706
:10367000E885F985C080D12CF4018085C81AD1086D
:10368000C901889F9001899F300D300D1124CC9C79
:10369000C001CD9C900D900D1124820F931F0E94AC
:1036A000D72F082F6091C00721E0620F08F46FEF59
:1036B000E981FA8181919191FA83E9830E9408302E
:1036C0007C0196014A855B85632D742D812FEC81E9
:1036D000FD810995362E472E182F7394B7CF209170
:1036E000BF07129F112D1124632D742D812F0E946D
:1036F0002030462F282F672FC5010E94742F539426
:1037000079CF822D0E9412302B960FB6F894DEBF2F
:103710000FBECDBFDF91CF911F910F91FF90EF9022
:10372000DF90CF90BF90AF909F908F907F905F90F1
:103730004F903F902F900895A0E0B0E0E2EAFBE1C7
:103740000C945235EC01809156010E949831092F5A
:10375000182F2091C00731E0230F08F42FEF30E03D
:1037600040E050E06FEF7FEF80E090E00E94FA359C
:103770007901101708F041C0C12ED12CF601E6588E
:10378000FD4F9081809157018923A9F19091C40741
:10379000915097FD15C0492F092E000C550BFA01C9
:1037A000EC53F84F81891813F3CF440F551FFA01DA
:1037B000EC53F84F218D328D2E153F0548F701C08F
:1037C00097016091C00741E0640F08F46FEFC901F1
:1037D0000E940830AC016091BD077091BE078091D6
:1037E000BF07FE0109950E942030462F282F672F22
:1037F000C6010E94742F1F5FBCCF802F0E94123021
:10380000CDB7DEB7E8E00C946E35A0E0B0E0EBE0B9
:10381000FCE10C9453358C01809156010E94983143
:10382000EC016091C0076695669521E0620F08F48F
:103830006FEF8091B8079091B9070E940830D82E99
:10384000CD17F0F4EC2EF12CF701E658FD4F9081E6
:1038500080915701892391F06091BD077091BE0757
:103860008091BF072D2D4C2FF80109950E94203023
:10387000462F282F672FC7010E94742FCF5FE0CFFC
:103880008D2F0E941230CDB7DEB7E7E00C946F3574
:10389000A0E0B0E0EEE4FCE10C944F356C018091C7
:1038A00056010E949831192FC82F6091C007669564
:1038B00066958091B8079091B9070E940830D82F7B
:1038C00080E48D0F0E94922F90E8F92EF80E8D2F34
:1038D0000E94922F20E8922E980EC11700F5AC2E70
:1038E000B12CF501E658FD4F908180915701892355
:1038F000A1F06091BD077091BE078091BF07ED2ECA
:103900000C2F292D4F2DF60109950E942030462FAE
:10391000282F672FC5010E94742FCF5FDECF812F24
:103920000E941230CDB7DEB7EBE00C946B35A0E00F
:10393000B0E0EDE9FCE10C944D355C01809156015D
:103940000E949831F92E182F6091C00766958091DA
:10395000B8079091B9070E940830782E1F1508F01B
:1039600043C0812E912CF401E658FD4F9081809147
:1039700057018923B9F1F401EE0FFF1FEA5DFD4FF6
:10398000C081D0E0C057D109F401EE0FFF1FEA500B
:10399000FE4FC1A8D12C80E2C81AD108CC9F90015B
:1039A000CD9F300D300D1124CC9CC001CD9C900DCD
:1039B000900D1124820F931F0E94D72F082F609122
:1039C000BD077091BE078091BF07E72C9601AE013D
:1039D000F50109950E942030462F282F672FC4013A
:1039E0000E94742F1F5FBACF8F2D0E941230CDB767
:1039F000DEB7EDE00C946935A0E0B0E0E2E0FDE177
:103A00000C9452357C01809156010E949831D92E38
:103A1000182F6091C00766958091B8079091B907FB
:103A20000E940830C82E1D1578F5C12FD0E0FE0188
:103A3000E658FD4F908180915701892319F1FE01CD
:103A4000EE0FFF1FEA50FE4F21A930E0205231094E
:103A5000FE01EE0FFF1FEA5DFD4F408150E0405731
:103A600051096091BD077091BE078091BF070C2D71
:103A7000F70109950E942030462F282F672FCE018D
:103A80000E94742F1F5FCFCF8D2D0E941230CDB7B3
:103A9000DEB7E8E00C946E35CF93DF93682F8A3061
:103AA00011F481E003C08D3021F480E00E94DC2419
:103AB0006FC08091B6079091B70726E0FC01A0EB9C
:103AC000B7E001900D922A95E1F7603E30F026E0D4
:103AD000FC0111922A95E9F70AC0F6E06F9FB00148
:103AE00011246658764F46E050E00E947F35C09121
:103AF000B607D091B70746E050E0BE0180EB97E0F3
:103B00000E944136892B49F19E01205B3340A90177
:103B100086E0569547958A95E1F781E090E0BC01F3
:103B200002C0660F771F4A95E2F74091AE035091AD
:103B3000AF03462B572B2B5F3F4F66E036952795FB
:103B40006A95E1F702C0880F991F2A95E2F7842B46
:103B5000952B9093AF038093AE039E012A5A334076
:103B60004091AD03642F70E0C9010E943435481BB9
:103B7000463010F4240F311D211584E0380710F071
:103B800020E030E020553C4F3093B7072093B60734
:103B9000DF91CF910895CF93DF93EC01FE018491E3
:103BA000882321F00E944C1D2196F8CFDF91CF9100
:103BB00008958091AB039091AC039C012C70332746
:103BC0002C30310511F4806101C08F7E0E94FB28EA
:103BD00008959091BC079370A1F0811102C0946088
:103BE00007C0803210F09C6703C0880F880F982BA5
:103BF0009093BC07109255018091AA038160809335
:103C0000AA0308959091BC07937071F08093BD074B
:103C10006093BE07453B08F044EB4093BF0780919B
:103C2000AA0381608093AA030895AAE2B0E0EBE1C1
:103C3000FEE10C945735E2EAF3E08AEA93E0209142
:103C4000F10021938E179F07D1F78091A303833052
:103C500009F461C030F4813071F0823009F49BC006
:103C6000B2C08A3009F487C08B3009F46CC0893047
:103C700009F0A9C020C08091A203813A09F0A3C035
:103C80008091E800877F8093E8008091A60390915F
:103C9000A703892B21F468E086E993E003C060E084
:103CA00080E090E070E00E9451238091E8008B77E3
:103CB0008093E80088C08091A203813209F083C01C
:103CC0008091A6039091A703029708F07CC0809191
:103CD000E800877F8093E8008091E80082FD05C0BE
:103CE0008091A0038111F8CF6EC02091F3008091E4
:103CF000F20090E0922B029731F48091F100813034
:103D000011F0863021F48091F10080939503809129
:103D1000E8008B7754C08091A203813A09F053C028
:103D20008091A6039091A703892B09F04CC0809144
:103D3000E800877F8093E8008091E80080FFFCCF57
:103D40008091540137C08091A2038132E1F58091C6
:103D5000A6039091A703892BB1F58091E800877F96
:103D60008093E8000E94CB218091A40380935401AA
:103D70000E94292928C08091A203813221F58091D7
:103D8000E800877F8093E8000E94CB218091A50303
:103D90008093940318C08091A203813AA1F480918A
:103DA000E800877F8093E8008091E80080FFFCCFE7
:103DB000809194038093F1008091E8008E77809346
:103DC000E8000E94CB218091E80083FFCEC1809162
:103DD000A2039091A303492F50E04A30510508F007
:103DE000C4C1FA01E258FF4F0C941936803821F013
:103DF000823809F0BAC108C080919E0390919F0358
:103E0000992389F082600FC08091A6038F7087305C
:103E100008F0ABC18093E9008091EB0085FB882717
:103E200080F91092E9009091E800977F9093E80064
:103E30008093F1001092F10065C1282F2D7F09F0C9
:103E400094C1882319F0823061F08FC18091A4035E
:103E5000813009F08AC1933009F080E080939F039C
:103E60002EC08091A40381112AC08091A6038F7077
:103E70002FEF280F263008F078C18093E9002091B9
